:020000040000FA
:1000000001288501860107309F0083160C3085008A
:10001000043086000130810083120508A300E2202D
:100020009820E220061D16288F201728FB205C2030
:10003000D6200508A30023192828A3192B288F20D0
:100040005C200508A300231D2128A31D21281828B2
:10005000A31D4428192827083F3C031919282608FE
:100060000F39031D36283530A60041283030A60050
:100070002508393C03193E28A50A41283030A5003F
:10008000A40AA70A5C20182827080319182826089C
:100090000F3903194E283030A60059283530A600F4
:1000A00025080F3903195628A50359283930A5000A
:1000B000A403A7035C2018280630A8002708A9007D
:1000C000A90DA90DA90D8501031805148514851026
:1000D000A80B6228850185178513AF202030BE202C
:1000E0007030BE206530BE203430BE203330BE209C
:1000F0003030BE203230BE202030BE20B220203032
:10010000BE202408BE202508BE202E30BE20260892
:10011000BE206430BE206230BE201621080033307D
:10012000A4003130A5003530A6003F30A7000800FC
:1001300006108610E2203030A200C720CD20E22039
:100140002030A200C720CD20E2202830B5200C307E
:10015000B5200630B5200130B520E22008008030FF
:10016000B5200800C030B5200800A2008610E820A5
:10017000C720CD20A20EC720CD200800A2008614E3
:10018000E820C720CD20A20EC720CD2008000F30C8
:1001900086052208F03986040800061400000610BF
:1001A000E82008000130B520E2200800F030A0006F
:1001B0000508A300231DDE28A31DDE28EA20A00BCE
:1001C000D82808000F30A000EA20A00BE42808007F
:1001D0001E30EB28FF30A1000000A10BEC28080026
:1001E0000230A100A10BF228080083169B001C140A
:1001F0001A08831208000130F520A4000230F5200F
:10020000A5000330F520A6000430F520A700080063
:1002100083168B131C1555309D00AA309D009C142D
:1002200083128C1F1029E2208C13080001308316E2
:100230009B008312240883169A000821023083163B
:100240009B008312250883169A0008210330831629
:100250009B008312260883169A0008210430831617
:100260009B008312270883169A0008211C11831211
:02027000080084
:02400E00103D63
:084202003300310035003F00DC
:00000001FF
